:1000000033C300004DC300004BC3000049C30000D0
:1000100047C3000045C3000043C3000041C30000C4
:100020003FC300003DC300003BC3000039C30000D4
:1000300037C3000035C3000033C3000031C30000E4
:100040002FC300002DC300002BC3000029C30000F4
:1000500027C3000025C300000C94B71021C3000083
:100060001FC300001DC300001BC3000019C3000014
:1000700017C3000015C3000013C3000011C3000024
:100080000FC300000DC300000C94731009C30000DF
:1000900007C3000005C3000003C3000001C3000044
:1000A000FFC20000FDC20000FBC20000F9C2000058
:1000B000F7C20000F5C20000F3C20000F1C2000068
:1000C000EFC20000EDC20000EBC20000E9C2000078
:1000D000E7C20000E5C20000E3C20000E1C2000088
:1000E000DFC20000DDC20000DBC20000D9C2000098
:1000F000D7C20000D5C20000D3C20000D1C20000A8
:10010000CFC20000CDC20000CBC20000C9C20000B7
:10011000C7C20000C5C20000C3C20000C1C20000C7
:10012000BFC20000BDC20000BBC20000B9C20000D7
:10013000B7C20000B5C20000B3C20000B1C20000E7
:10014000AFC20000ADC20000ABC200000C945B1156
:10015000A7C20000A5C20000A3C20000A1C2000007
:100160009FC200009DC200009BC2000099C2000017
:1001700097C2000095C2000093C2000091C2000027
:100180008FC200008DC200008BC2000089C2000037
:1001900087C2000085C2000083C2000081C2000047
:1001A0007FC200007DC200007BC2000079C2000057
:1001B00077C2000075C2000073C2000071C2000067
:1001C0006FC200006DC200006BC2000069C2000077
:1001D00067C2000065C2000063C2000061C2000087
:1001E0005FC200005DC200005BC2000059C2000097
:1001F00057C200000C941B2153C200001C034C008A
:100200005500460041002000430044004300200008
:10021000440065006D006F00000018034400650095
:1002200061006E002000430061006D0065007200F7
:10023000610000000403090409023E00020100C03D
:10024000320904000001020201000524001001042B
:100250002402060524060001070582030800FF09A1
:10026000040100020A00000007050402100005074F
:100270000583021000051201100102000008EB03C3
:10028000442001000102DC01004E4F4E45000000F9
:10029000000000000000000000400441044204434C
:1002A00004440445044804490400000001014D468B
:1002B0005F434C41535349435F314B0000004C12A4
:1002C000831201131B131F1320139D17A317000480
:1002D0000400024D465F434C41535349435F344B46
:1002E0000000004C1283120E131B131F1320139DCA
:1002F00017A317001004004E4F4E450000000000E9
:1003000000000000000000000000000000000000ED
:10031000000000000000005549445F52414E444F28
:100320004D00000000000000000000000000000080
:10033000000000000000005549445F4C4546545FF2
:10034000494E4352454D454E540000000000000008
:10035000000000000000005549445F5249474854DE
:100360005F494E4352454D454E5400000000000089
:10037000000000000000005549445F4C4546545FB2
:1003800044454352454D454E5400000000000000D6
:10039000000000000000005549445F52494748549E
:1003A0005F44454352454D454E5400000000000057
:1003B000000000000000004359434C455F53455482
:1003C00054494E47530000000000000000000000A8
:1003D000000000000000004368616D656C656F6E91
:1003E0002D4D696E69202553207573696E67204C09
:1003F00055464120255320636F6D70696C656420FC
:1004000077697468204156522D4743432025530095
:100410003134303531310031333039303100342E20
:10042000372E320025730052414E444F4D00257542
:1004300000257500253575206D56005645525349E7
:100440004F4E000000000000000000000000003AD5
:100450000B434F4E464947000000000000000000DB
:1004600000760B6E0B580B5549440000000000004D
:10047000000000000000000000A10B7B0B52454172
:10048000444F4E4C59000000000000000000000ADC
:100490000CF80B55504C4F41440000000000000088
:1004A0000000001E0C00000000444F574E4C4F410E
:1004B000440000000000000000230C000000005277
:1004C00045534554000000000000000000000028D3
:1004D0000C00000000555047524144450000000008
:1004E0000000000000330C000000004D454D534952
:1004F0005A45000000000000000000000000003E1F
:100500000C55494453495A450000000000000000C2
:100510000000000000560C425554544F4E0000009D
:10052000000000000000006C0C760C710C53455468
:1005300054494E4700000000000000000000008306
:100540000C7E0C434C4541520000000000000000AE
:100550000000008B0C0000000048454C50000000DB
:100560000000000000000000008E0C00000000529F
:10057000535349000000000000000000000000008C
:10058000000000DA0C000000000000000000000085
:1005900000000000000000000000000D0A000D0A2D
:1005A00000643130303A4F4B000000000000000082
:1005B000000000000000000000000000000000003B
:1005C0000000653130313A4F4B2057495448205490
:1005D000455854000000000000000000000000002A
:1005E0000000006E3131303A57414954494E47209E
:1005F000464F5220584D4F44454D0000000000002A
:1006000000000000C83230303A554E4B4E4F574E26
:1006100020434F4D4D414E440000000000000000BB
:100620000000000000C93230313A494E56414C4971
:100630004420434F4D4D414E4420555341474500C2
:10064000000000000000CA3230323A494E56414C98
:10065000494420504152414D45544552000000004C
:10066000000000000000000011241FBECFEFDFE2F9
:10067000DEBFCDBF10E2A0E0B0E2E0EFFEE402C0DA
:1006800005900D92A239B107D9F726E2A2E9B0E2AE
:1006900001C01D92AD39B207E1F703D00C94762763
:1006A00078C07DD0AED680E38093010627D20DD1ED
:1006B0006DD781D135D581E080930002109201027F
:1006C00092E09093020293E09093040280932002C0
:1006D00088E380932102CED0C1E05DD7E091EB208A
:1006E000F091EC200995E091F120F091F22009952C
:1006F00080910C0A80FFF1CFC0930C0A6FD16AD7AA
:1007000016D5809193208093060610929320E5CF12
:10071000292F33272230310539F123303105A9F053
:100720002130310549F020E030E080E090E0FA012E
:1007300080839183C901089522E130E086E792E049
:10074000FA0180839183C901089599278130910529
:10075000A1F082309105B9F0892B29F7E4E3F2E0AA
:10076000249130E0CF01E3CF2EE330E088E392E044
:10077000FA0180839183C9010895EAE1F2E02491AE
:1007800030E0CF01D4CFECEFF1E0249130E0CF01A5
:10079000CECF1F920F920FB60F921124FFCF8091F0
:1007A000780083FF0AC088E08093780088ED84BFDA
:1007B00081E080938000FD95FEC0809150008660AE
:1007C000809350008091510081FFFCCF80915100B7
:1007D00082FFFCCF1092560021E02093600088ED4C
:1007E00084BF2093400083ED90E38093260A90938A
:1007F000270A86E08093000A209343002093000498
:100800008091CC0188608093CC01089588ED84BFED
:1008100081E0E8E7F0E08183089588ED84BF8BE113
:100820008093800008958BEC80935200809150005B
:100830008860809350008091510083FFFCCF84EC4E
:10084000809355008091500080618093500080918A
:10085000510084FFFCCF0895E0E4F0E084818E7FB6
:100860008483E0E5F0E080818F7E80838081877FD4
:100870008083089587E0E0EAF0E082837894089529
:100880000895089508950895089580E090E00895EA
:1008900008950895E091FE20F091FF20818395E274
:1008A000899FB001112468577D4F45E250E088EDE3
:1008B00090E20E940D24E091ED20F091EE20099548
:1008C000E091E920F091EA200994E091FE20F09176
:1008D000FF208181DFCF0F931F93CF93DF9320E021
:1008E00030E015E2AC014F5F5F4F022F129FF00125
:1008F000139FF00D1124E757FD4F649161110FC054
:10090000EC016881662301F12F5F3F4F23303105F1
:1009100061F780E0DF91CF911F910F910895DC0185
:100920007C91772389F36713EFCFDA0105C07D91BE
:10093000772351F37613E8CF3196ED01649161117D
:10094000F6CF68816111E0CF802FA4DF81E0DF91D5
:10095000CF911F910F910895CF93DF93EC016150D8
:10096000710980E090E035E24CE2389FF001399F58
:10097000F00D1124E757FD4F2491222381F06131BE
:10098000710568F0DE0103C06031710541F02D93FF
:10099000ED0131966150710924912111F5CF82301A
:1009A000910521F41882DF91CF9108954993615008
:1009B00071090196DACF08950C94FF2308951F93CF
:1009C000CF93DF93162F662329F0EC01F5DF89938F
:1009D0001150E1F7DF91CF911F9108950E94FF23FD
:1009E0000E94FF230E94FF230C94FF23CF93DF93E9
:1009F000DC01615071092115310599F162307105F1
:100A000080F1FA01240F351F2150310940E050E0F8
:100A100017C0D05DDC93CF708C2F90E00A97FCF468
:100A2000C05D1196CC9311971296625071094E5F7A
:100A30005F4FE217F307B9F031966230710598F015
:100A4000C081DC2FD295DF708D2F90E00A970CF3D8
:100A5000D95CDC93CF708C2F90E00A970CF3C95CC3
:100A6000E0CF40E050E01C92CA01DF91CF910895A1
:100A7000FA0140814423F1F151815523D9F16115E7
:100A80007105C1F1DC0120E030E013C04295407FE8
:100A9000513428F5582F452B4D932F5F3F4F3296F9
:100AA0004081442329F15181552321F162177307B5
:100AB000F9F0842F80538A3018F081518630D0F4B9
:100AC000852F80538A3020F0952F9154963090F4E2
:100AD0004134E0F24295407F40575134D8F25753A9
:100AE000452B4D932F5F3F4F329640814111DBCF15
:100AF000C901089520E030E0C9010895CF93DF9344
:100B000000D000D0CDB7DEB780E18093650692E0DB
:100B10009093660698E0909365069AE1909361063B
:100B20001092A6091092A70990EC9093A50998E15C
:100B30009093A4098093660687ED8093A009809125
:100B4000A10986FFFCCF80E48093A1098091A009D0
:100B50001092A0098091A10986FFFCCF80E48093C8
:100B6000A1098091A00990E19093650680FD3EC0A7
:100B70008DE389838AE28A8380E88B8386EA8C838B
:100B800020E137ED90E4209366063093A009809130
:100B9000A10986FFFCCF9093A1098091A009109232
:100BA000A0098091A10986FFFCCF9093A1098091B3
:100BB000A0092093650687FFE6CF80E18093660653
:100BC000FE013196CE01059630E421912093A009D3
:100BD0002091A10926FFFCCF3093A1092091A00903
:100BE000E817F90791F780E1809365062496CDBF59
:100BF000DEBFDF91CF910895CF92DF92EF92FF9207
:100C00000F931F93FC010091FD2010E020E030E0E5
:100C1000980111270027060F171F211D311D60E1C4
:100C200077ED90E4609366067093A0098091A10926
:100C300086FFFCCF9093A1098091A0091092A00992
:100C40008091A10986FFFCCF9093A1098091A00912
:100C50006093650687FFE6CF80E18093660683E0B8
:100C60008093A0098091A10986FFFCCF80E4809346
:100C7000A1098091A0096901EE24FF24C092A00976
:100C80008091A10986FFFCCF80E48093A109809127
:100C9000A009C12ED22EE32EFF24C092A00980917C
:100CA000A10986FFFCCF80E48093A1098091A0096F
:100CB0000093A0098091A10986FFFCCF80E4809376
:100CC000A1098091A0094115510589F04E0F5F1FC0
:100CD00090E41092A0098091A10986FFFCCF909327
:100CE000A1098091A0098193E417F50791F780E1AC
:100CF000809365061F910F91FF90EF90DF90CF904A
:100D000008954F925F926F927F928F929F92AF92CF
:100D1000BF92CF92DF92EF92FF920F931F93CF93E8
:100D2000DF939C01FA018091FD2090E0A0E0B0E00B
:100D3000DC0199278827860F971FA11DB11D3097C9
:100D400009F411C1E12CFF24F39410E1C12E07ED49
:100D5000B02E40E4D42E50E1A52E67ED962E73E51B
:100D6000472EC4E85C2ED3E86D2E492F5A2F6B2FE7
:100D70007727852ED82F8701081B1109E017F10767
:100D800008F48F01A09266069092A009C091A10973
:100D9000C6FFFCCFD092A109C091A0091092A00972
:100DA000C091A109C6FFFCCFD092A109C091A009B2
:100DB000C0926506C7FFE6CFA09266064092A009E2
:100DC000C091A109C6FFFCCFD092A109C091A00992
:100DD0008092A009C091A109C6FFFCCFD092A109C1
:100DE000C091A009742E4093A0094091A10946FF2B
:100DF000FCCFD092A1094091A0091092A009409186
:100E0000A10946FFFCCFD092A1094091A009C09250
:100E10006506C0926606B092A0094091A10946FFFE
:100E2000FCCFD092A1094091A0091092A009409155
:100E3000A10946FFFCCFD092A1094091A009C09220
:100E4000650647FFE6CFA09266065092A009409142
:100E5000A10946FFFCCFD092A1094091A0091092B0
:100E6000A0094091A10946FFFCCFD092A109409171
:100E7000A0091092A0094091A10946FFFCCFD09291
:100E8000A1094091A009D093A0094091A10946FF72
:100E9000FCCFD092A1094091A0090115110591F054
:100EA000A901400F511FE90169916093A009609168
:100EB000A10966FFFCCFD092A1096091A009C417D7
:100EC000D50791F7C0926506C0926606B092A00958
:100ED0004091A10946FFFCCFD092A1094091A00901
:100EE0001092A0094091A10946FFFCCFD092A10920
:100EF0004091A009C092650647FFE6CFA092660622
:100F00006092A0094091A10946FFFCCFD092A109AF
:100F10004091A0098092A0094091A10946FFFCCF11
:100F2000D092A1094091A0097092A0094091A10915
:100F300046FFFCCFD092A1094091A0091092A009D0
:100F40004091A10946FFFCCFD092A1094091A00990
:100F5000C0926506E01BF10B800F911FA11DB11D12
:100F6000309709F002CFDF91CF911F910F91FF9041
:100F7000EF90DF90CF90BF90AF909F908F907F9039
:100F80006F905F904F9008958091FD2090E0A0E0D9
:100F9000B0E0BA2FA92F982F88279C01339560E1E4
:100FA00077ED50E4E1E8609366067093A009409104
:100FB000A10946FFFCCF5093A1094091A0091092CE
:100FC000A0094091A10946FFFCCF5093A10940918F
:100FD000A0096093650647FFE6CF60936606E0933D
:100FE000A0094091A10946FFFCCF5093A10940916F
:100FF000A0099093A0094091A10946FFFCCF50930E
:10100000A1094091A0098093A0094091A10946FF40
:10101000FCCF5093A1094091A0091092A0094091E2
:10102000A10946FFFCCF5093A1094091A00960930C
:10103000650601968217930709F0B5CF0895CF9200
:10104000DF92EF92FF920F931F93FC01CB01BA0145
:1010500069016115710521E08207910540F081E089
:101060001F910F91FF90EF90DF90CF90089500E0D7
:1010700010E021E030E0061B170B280B390BE12CA8
:10108000F12C0C151D052E053F0558F0A601CF01CA
:1010900038DE81E01F910F91FF90EF90DF90CF90AD
:1010A000089568017901A601CF012BDEF2CFCF921E
:1010B000DF92EF92FF920F931F93FC01CB01BA01D5
:1010C00069016115710521E08207910540F080E01A
:1010D0001F910F91FF90EF90DF90CF90089500E067
:1010E00010E021E030E0061B170B280B390BE12C38
:1010F000F12C0C151D052E053F0558F0A601CF015A
:101100007BDD81E01F910F91FF90EF90DF90CF90FA
:10111000089568017901A601CF016EDD81E0F2CF6B
:10112000E0E0F6E080E4828388E1868B0895FF9218
:101130000F931F93CF93DF93CDB7DEB7A097CDBFAB
:10114000DEBF809108068095909192209827809329
:10115000922080748923A9F0E091FE20F091FF2075
:1011600080818130B9F0823079F1833009F44EC04A
:10117000843009F46FC0853009F48EC0863009F4DC
:1011800067C0A096CDBFDEBFDF91CF911F910F91B9
:10119000FF9008958091FB20882309F49FC0F12CD3
:1011A0008E010F5F1F4F08DCF801EF0DF11D8083EA
:1011B000F3948091FB20F816B0F3E091F720F091C2
:1011C000F820C8010995DDCFE091F520F091F620D7
:1011D0008E010F5F1F4FC80109952091FB2022232C
:1011E00061F3F801CE0102962150820F911D21E09A
:1011F000222339F0308121E03F3F09F020E03F5FBA
:1012000030833196E817F90799F7D7CFE091F520A9
:10121000F091F6208E010F5F1F4FC80109952091B4
:10122000FB2031E0215048F23323E1F3822F90E09C
:10123000F801E80FF91F408131E04F3F09F030E03D
:10124000F801E80FF91F4F5F4083215068F7B5CFD1
:10125000F7D097CFE091F520F091F6208E010F5F47
:101260001F4FC80109952091FB20222309F4A5CF27
:10127000F801CE0102962150820F911D21E0222318
:1012800031F0308121E0311120E03150308331964E
:10129000E817F907A1F791CFE091F520F091F6203A
:1012A0008E010F5F1F4FC80109952091FB2031E08F
:1012B000215008F482CF3323D9F3822F90E0F80134
:1012C000E80FF91F408131E0411130E0F801E80FEB
:1012D000F91F41504083215070F76FCF8E010F5F8F
:1012E0001F4F6BCFCF93DF93EC016150710980E00A
:1012F00090E03CE2FC01EE0FFF1FE295F295F07FDB
:10130000FE27E07FFE27E950FD4F2491222381F044
:101310006132710568F0DE0103C06032710541F091
:101320002D93ED0131966150710924912111F5CF72
:101330008630910521F41882DF91CF910895399379
:10134000615071090196D6CFE091FE20F091FF2007
:1013500080830895AB01E091FE20F091FF20608131
:1013600020E2629FB001112469507D4F0C941F242C
:10137000CF93DF93EC0167EF72E00E941624892B74
:1013800071F167E173E0CE010E941624892B69F1A7
:1013900067E373E0CE010E941624892B41F167E5D3
:1013A00073E0CE010E941624892B19F167E773E0E0
:1013B000CE010E941624892BF1F067E973E0CE017B
:1013C0000E941624892BC9F067EB73E0CE010E94BE
:1013D0001624892BA1F080E0DF91CF91089580E061
:1013E000B3DF81E0DF91CF91089581E0F9CF82E012
:1013F000F7CF83E0F5CF84E0F3CF85E0F1CF86E04F
:10140000EFCF43E150E060E070E08DEF90E20C94AC
:10141000312643E150E060E070E08DEF90E20C9403
:101420003C26883008F008958093FD2090E0880FD6
:10143000991F80509F4D8093FE209093FF2045CAB6
:101440002091FD2030E02F5F3F4F27703327822F00
:10145000F901EE0FFF1FEF5FFE4D908191115CC00F
:101460002F5F3F4F27703327822FF901EE0FFF1FA9
:10147000EF5FFE4D908191114FC02F5F3F4F27705E
:101480003327822FF901EE0FFF1FEF5FFE4D908192
:10149000911142C02F5F3F4F27703327822FF901F0
:1014A000EE0FFF1FEF5FFE4D9081911135C02F5F52
:1014B0003F4F27703327822FF901EE0FFF1FEF5F99
:1014C000FE4D9081911128C02F5F3F4F2770332729
:1014D000822FF901EE0FFF1FEF5FFE4D90819111FA
:1014E0001BC02F5F3F4F27703327822FF901EE0F6C
:1014F000FF1FEF5FFE4D908191110EC02F5F3F4F98
:1015000027703327822FF901EE0FFF1FEF5FFE4D8B
:101510009081911101C0089584CF8091FD2008959C
:10152000CF93DF93EC01F9DF805D88831982DF912F
:10153000CF910895FC0180819181911103C0805366
:10154000883010F080E008956CDF81E00895BC01E0
:1015500080E090E20C94AD21CF93DF93EC012196D3
:10156000FC016491662349F080E090E20E94002231
:10157000FE01219664916111F7CFDF91CF9108951B
:10158000AB01BC0180E090E20C94D62180E2E0E661
:10159000F6E082830895CF93DF9380E090E20E948B
:1015A0007F220E94801C80E090E20E949A22EC013F
:1015B00097FD09C080E180939320809305068C2FCE
:1015C00062D2882319F0DF91CF9108958C2FDF919B
:1015D000CF91C9C380919420813001F130F08230E5
:1015E00059F1833071F091D35FC58091680685FF12
:1015F000FACF84E180931B2081E08093942085D3EF
:1016000053C580911B20815080931B208111EBCF0B
:101610000E94AA2021D910929420E5CF80911B200E
:10162000815080931B208111DECFFDD80E94E520E0
:1016300082E080939420D7CF8091680685FDD3CF38
:1016400084E180931B2083E0809394205ED32CC59B
:1016500080E2E0E0F6E08583089580E2E0E0F6E0F5
:101660008683089580E090E20C94882180E090E2E7
:101670000C94FA222EE134E03F932F9327E134E0DB
:101680003F932F9320E134E03F932F9327ED33E0F6
:101690003F932F9321E02F931F929F938F930E944C
:1016A00037248DB79EB70C968DBF9EBF85E60895F3
:1016B00029ED30E23F932F9324E234E03F932F93C0
:1016C00021E02F931F929F938F930E9437248DB711
:1016D0009EB708968DBF9EBF85E60895FCD8811100
:1016E00002C08AEC089595DE84E6089560E071E01A
:1016F00033D985E608950F931F93CF93DF93CDB72A
:10170000DEB7A197CDBFDEBF8C012091FB20E09119
:10171000F520F091F620CE01019629A3099529A183
:1017200030E0AE014F5F5F4F60E071E0C8015ED90D
:1017300085E6A196CDBFDEBFDF91CF911F910F91BE
:101740000895BF92CF92DF92EF92FF920F931F9373
:10175000CF93DF93CDB7DEB7A097CDBFDEBF8C01AF
:10176000C090FB20D12C67E274E00E941624892BE4
:1017700051F5C114D104B1F1B12CEE24E394F12C54
:10178000EC0EFD1E00E010E017D9F701E00FF11F8D
:101790008083B3940B2D10E00C151D05A8F3E09188
:1017A000F720F091F820C701099584E6A096CDBFF7
:1017B000DEBFDF91CF911F910F91FF90EF90DF90EF
:1017C000CF90BF900895A80160E270E0EE24E3940A
:1017D000F12CEC0EFD1EC7014BD98C159D05F9F2BD
:1017E0008AECE4CFEE24E394F12CEC0EFD1ED7CF6F
:1017F0002091FC20211107C020E3FC012083FC0183
:10180000118285E6089521E3FC012083FC01118209
:1018100085E60895FC012181211105C08081813375
:1018200041F0803311F08AEC08951092FC2084E698
:10183000089581E08093FC2084E608958FE198E08C
:10184000F7D08EE6089587E598E00AD18EE60895F0
:10185000E0ECF4E081818E7F81830E94AA200E94C7
:10186000060484E60895E0ECF4E081818E7F8183B4
:101870000E94AA200E940D0484E60895E9EFF0E298
:1018800021812F9320812F932EE234E03F932F93D9
:1018900021E02F931F929F938F930E9437248DB73F
:1018A0009EB708968DBF9EBF85E608952091FB20C8
:1018B0001F922F9321E334E03F932F9321E02F9346
:1018C0001F929F938F930E9437248DB79EB70896DF
:1018D0008DBF9EBF85E6089560E071E003DD85E67B
:1018E000089560E071E036DD85E6089541DD8111FF
:1018F00002C08AEC08958DDD84E6089560E071E011
:101900000FDE85E6089516DE811102C08AEC089587
:1019100080DD84E6089538DB84E60895BF92CF9297
:10192000DF92EF92FF920F931F93CF93DF937C018F
:10193000CFEFD0E03BE3C32E34E0D32E4CE2B42E05
:101940008601B60180E990E20E941624892B21F1DC
:10195000F6018491882389F0C132D10570F0D70156
:1019600003C0C032D10549F08D937D010F5F1F4F39
:101970002197F80184918111F4CFF701B1927F0191
:101980002197F6E1CF0ED11C8601B60180E990E2E5
:101990000E941624892BE1F6F7013197108285E623
:1019A000DF91CF911F910F91FF90EF90DF90CF903B
:1019B000BF900895FC01209120022068209320020E
:1019C0002091230220FFFCCF81E080932302A0918D
:1019D0001002B0911102AE5BB109B7FD1CC029E63F
:1019E00037E54BE050E00E949723AA27BB279F933F
:1019F0008F9324E334E03F932F9381E08F931F92E2
:101A0000FF93EF930E9437248DB79EB708968DBF42
:101A10009EBF85E60895A0E0B0E0E1CF80E0E0E180
:101A2000F1E29191890F91E2E039F907D1F7089538
:101A300021E0209395202093962024E12093972065
:101A400025E0209398201092992010929A201092CD
:101A50009B2010929C2080939D2090939E2008951F
:101A600027E02093952024E6209398201092992037
:101A700010929A2010929B2010929C2080939D207F
:101A800090939E200895CF93C82F909195209530E4
:101A900009F47FC0E0F0973009F44AC060F5209166
:101AA000A22080919620281709F4DFC030E090E052
:101AB00001972817390709F407C168E180E090E22F
:101AC0000E9400221092952081E0CF9108959330DA
:101AD00009F457C0B8F090E04091A2202FEF30E019
:101AE000241B31098217930709F06AC085E08093AF
:101AF000952081E0EACF9830F1F09930A1F080E0B4
:101B0000CF9108959130D8F3813009F4DFC084304B
:101B100029F0883141F081E0CF91089566E080E0BE
:101B200090E20E9400221092952081E0CF910895CA
:101B3000853109F450C0C83189F3C63009F4E1C0D9
:101B4000C53149F761E080E090E20E940022609197
:101B5000962080E090E20E9400226091962060959D
:101B600080E090E20E94002260E870E080E191E273
:101B700007DD54DF682F80E090E20E94002281E0C0
:101B8000A4CF8093A22084E08093952081E0CF9120
:101B9000089520919F203091A020F901E05FFE4D33
:101BA0008083C901019680939F209093A020803864
:101BB000910509F0B0CF86E08093952081E085CF34
:101BC00065E180E090E20E94002282E0809395200F
:101BD00081E0CF91089581E08093962040919920F3
:101BE00050919A2060919B2070919C20E0919D20C3
:101BF000F0919E2020E830E080E191E20995882371
:101C000009F46FC061E080E090E20E9400226091E0
:101C1000962080E090E20E940022609196206095DC
:101C200080E090E20E94002260E870E080E191E2B2
:101C3000A7DCF4DE682F80E090E20E940022809111
:101C4000992090919A20A0919B20B0919C2080583F
:101C50009F4FAF4FBF4F8093992090939A20A093AE
:101C60009B20B0939C2081E057CFD8DE8C13A8CF67
:101C70004091992050919A2060919B2070919C20D6
:101C8000E0919D20F0919E2020E830E080E191E2FB
:101C90000995882381F1809196208F5F809396200B
:101CA0008091992090919A20A0919B20B0919C20A6
:101CB00080589F4FAF4FBF4F8093992090939A20A9
:101CC000A0939B20B0939C2066E07BCF10929F2036
:101CD0001092A0201092A12083E08093952081E0B3
:101CE000F4CE64E080E090E20E94002289E08093DC
:101CF000952081E0EACE68E180E090E20E94002237
:101D0000DCCE809196208F5F67CF809195208130C7
:101D100071F0873009F0089580919820982F9150A4
:101D2000909398208111F7CF10929520089580917B
:101D30009820982F9150909398208111ECCF80910A
:101D40009720982F915090939720811106C0109260
:101D5000952085E080939820089565E180E090E2E9
:101D60000E940022F6CF1F93CF93DF93982F9154B8
:101D70009A3120F090529A31B8F480522091A320E9
:101D80003091A4202F3F310550F4F901E05FFE4D62
:101D900080832F5F3F4F2093A3203093A42081E0C6
:101DA000DF91CF911F9108959F5C9A3038F38F3562
:101DB00029F38F3319F38D3309F38D30A9F088306F
:101DC00039F08B3161F71092A3201092A420E7CF55
:101DD0008091A3209091A420009709F3019780930C
:101DE000A3209093A420DBCFE091A320F091A42026
:101DF000E05FFE4D10821092A3201092A4208091EB
:101E00001021882309F4A2C08F3309F49FC08D33B9
:101E100009F49CC0E1E1F1E204C01F3331F01D334D
:101E200021F0EF0111911111F8CF18826BE374E0EA
:101E300080E191E20E941624892B09F432C161E508
:101E400074E080E191E20E941624892B09F426C1F6
:101E500067E674E080E191E20E941624892B09F480
:101E60001AC16DE774E080E191E20E941624892B8B
:101E700009F40EC163E974E080E191E20E94162446
:101E8000892B09F402C169EA74E080E191E20E94C1
:101E90001624892B09F4F6C06FEB74E080E191E21F
:101EA0000E941624892B09F4EAC065ED74E080E1F4
:101EB00091E20E941624892B09F4DEC06BEE74E0D7
:101EC00080E191E20E941624892B09F4D2C061E0DE
:101ED00075E080E191E20E941624892B09F4C6C0C6
:101EE00067E175E080E191E20E941624892B09F4F4
:101EF000BAC06DE275E080E191E20E941624892B60
:101F000009F4AEC063E475E080E191E20E9416241A
:101F1000892B09F4A2C069E575E080E191E20E9495
:101F20001624892B09F496C06FE675E080E191E2F2
:101F30000E941624892B09F48AC065E875E080E1C7
:101F400091E20E941624892B09F452C088ECC0E06B
:101F5000E1EAF5E0E4918E1709F430C0E2ECF5E037
:101F6000E4918E1709F441C0E3EEF5E0E4918E1799
:101F700009F438C0E4E0F6E0E4918E1781F1E5E27F
:101F8000F6E0E4918E1741F1E6E4F6E0E4918E1775
:101F900001F180E090E0E0DA8BE995E0DDDACC2336
:101FA00009F4FDCE80911021882309F4F8CE80E158
:101FB00091E2CDDA8EE995E0CFDAF1CE20E030E0A3
:101FC00041E2429FC001439F900D11248E559A4FCC
:101FD000E2CF25E030E0F4CF24E030E0F1CF23E0A1
:101FE00030E0EECF22E030E0EBCF21E030E0E8CF90
:101FF0002FE030E01092102146E1429FC001439F44
:10200000900D1124855C9B4F1F33F9F01D3389F02F
:10201000112319F089ECC1E09BCF4096FC0185911A
:102020009491FC010097B1F380E191E20995C1E040
:102030008FCF4296FC0185919491FC01009751F35A
:10204000CE0101960995C1E083CF4496E7CF2EE0FB
:1020500030E0D0CF2DE030E0CDCF2CE030E0CACF63
:102060002BE030E0C7CF2AE030E0C4CF29E030E0F9
:10207000C1CF28E030E0BECF27E030E0BBCF26E084
:1020800030E0B8CF25E030E0B5CF24E030E0B2CF8B
:1020900023E030E0AFCF22E030E0ACCF21E030E011
:1020A000A9CF20E030E0A6CF0895A0E2B6E082E01C
:1020B00011968C93119715968C931597E0E4F8E0A0
:1020C00010A211A28DE291E086A397A38FEF9FEF5C
:1020D00080A791A781E0808398E8938393E097831A
:1020E0001A968C9308951F920F920FB60F92112497
:1020F0008F939F93EF93FF9380E192E28093B120BF
:102100009093B22080E992E28093B3209093B42020
:102110001092AA201092A9201092A5201092AD2012
:102120001092AE201092A820E0E4F8E0138286E935
:1021300090E086AB97AB8AE190E080AF91AFE0E4AE
:10214000F9E010A211A28FEF9FEF86A397A389E871
:1021500083838EE08083E0E2F6E01286FF91EF91C8
:102160009F918F910F900FBE0F901F9018951F9207
:102170000F920FB60F9211242F938F939F93EF938B
:10218000FF93909128068091A920957021E009F095
:1021900020E0880F822B8093A9209091A52099237D
:1021A000A1F1982F9770973009F442C0982F9C7036
:1021B00061F191E082FD6BC09093A7208091A820EF
:1021C00081116DC08091AA208695992309F471C070
:1021D00020E8282B2093AA208091AD209091AE205A
:1021E00001968093AD209093AE2087709927892B1C
:1021F00061F4E091B120F091B2202193E093B120FD
:10220000F093B22081E08093A8208091A52091E0F6
:1022100089278093A52088E880934308FF91EF9158
:102220009F918F912F910F900FBE0F901F90189537
:102230001092400880E180934C08109243098091ED
:10224000A720882379F18CEB94E080936609909322
:1022500067091092A62081E080934C0983E0809367
:1022600046098091AD209091AE20877061F09091E9
:10227000AA208F5F96958F5F8930E1F7E091B120BA
:10228000F091B220908381E08093AF20BECF90E0A8
:102290009093A7208091A820882309F493CF1092CF
:1022A000A820B3CF8CE794E08093660990936709E8
:1022B000D0CF20E08ECF1F920F920FB60F92112435
:1022C0002F933F938F939F93EF93FF938091A6203B
:1022D000853009F44DC0A8F0883009F47CC020F5A1
:1022E000863009F4B8C0873009F48AC0FF91EF91B5
:1022F0009F918F913F912F910F900FBE0F901F9044
:102300001895823071F1F8F0833009F456C08430AA
:1023100069F78091AA2080FDB7C080E480934606CB
:1023200085E08093A620E2CF893009F45BC08A3033
:10233000E9F610924009109246091092000881E0D7
:102340008093B020D3CF882309F453C0813071F635
:102350008FE390E080936609909367098EE0809305
:10236000000880E48093450683E08093A620BECFDA
:102370008091AA2090E480FD84C0909345068695C4
:102380008093AA208091AB209091AC2001968093FD
:10239000AB209093AC209C0127703327232B09F4AA
:1023A00077C02091AD203091AE208217930709F0BD
:1023B0004EC088E08093A62099CF80E480934606A3
:1023C00084E08093A620E091B120F091B22080813A
:1023D0008093AA208BCF80E48093460689E0809387
:1023E000A62084CF80E4809346068AE08093A620CE
:1023F0007DCF8FE790E0809366099093670976CF51
:10240000E091B320F091B4208081811136C080E446
:10241000809345062091AB203091AC208091AD2077
:102420009091AE202817390721F23196E093B3201E
:10243000F093B420E091B120F091B220CF01019649
:102440008093B1209093B22081818093AA2084E070
:102450008093A6204BCFE091B320F091B4208081EF
:10246000811107C080E48093460687E08093A62010
:102470003DCF80E480934506F8CF80E48093460604
:10248000C9CF909346067BCF80E48093450648CF22
:1024900086E08093A6202ACFCF93DF93E0E4F6E096
:1024A00084E08283128AC0E8D1E082E68E83A0E2D3
:1024B000B6E085E012968C93129781E050968C934B
:1024C000509782E052968C9352971A961C921A97C4
:1024D00083E019968C9398E598839AE5998390E424
:1024E0009183968381838683E0E0F8E08FE090E03B
:1024F00086A397A388E090E082A793A783E28183D5
:10250000DF91CF91D2CDCF93DF938091AF208823FD
:10251000C1F01092AF2082E08093210680932606BE
:102520006091AD207091AE206115710589F4E09144
:10253000EF20F091F0200995109240091092460981
:10254000B4DD8091B02081112AC0DF91CF91089530
:10255000E091F320F091F42080E192E2099594FF5C
:1025600023C09F7E009741F38093AD209093AE20CF
:102570001092AB201092AC2080E192E28093B120C7
:102580009093B22080E992E28093B3209093B4209C
:1025900081E08093A6208091B0208823B1F2109230
:1025A000B020DF91CF9181CDAC01569547955695DE
:1025B00047955695479541155105A1F260E020E0F9
:1025C00030E0F901E05FFD4D2081022E22952025AB
:1025D000022E269526952025E058FF4F30E02F5FEC
:1025E0003F4F21FB772770F9C72F20E0D22F71E0F2
:1025F000C727C0836F5F262F30E02417350708F305
:10260000B1CF81E08093B52084E090E08093B62044
:102610009093B72088E08093B820089581E080935C
:10262000B52082E090E08093B6209093B72088E1B7
:102630008093B820089581E08093B520089508958F
:102640006F927F928F929F92AF92BF92CF92DF92C2
:10265000EF92FF920F931F93CF93DF93CDB7DEB727
:102660002E97CDBFDEBF8C018091B520843009F458
:10267000F4C008F43BC0863009F4BDC008F060C067
:10268000F801D08031D78D25D8018C931196DC903C
:102690002BD78D25F8018183D28026D78D25D801AF
:1026A00012968C9312971396DC901ED78D25F80105
:1026B00083838081803309F4ACC2803A09F41FC35C
:1026C000803C09F43AC3813C09F4DAC3823C09F442
:1026D000E7C3803B09F4F1C38056823008F494C10B
:1026E00081E08093B52020E030E063C0823009F4BF
:1026F000A0C008F471C0F8018081863209F46FC16E
:10270000823509F46CC1803509F474C1982F905654
:10271000923008F4E6C1803351F0803A41F0803CB9
:1027200031F0813C21F0823C11F0803BC9F681E020
:102730008093B52084E0F801808324E030E039C044
:102740008A3008F055C0D801FC90CED68F25F8010C
:102750008083F180C9D68F25D80111968C9311976B
:102760001296FC90C1D68F25F8018283F380BCD6E7
:102770008F25D80113968C9313971496FC90B4D69A
:102780008F25F8018483F580AFD68F25D801159663
:102790008C9364E070E0C80125D481110CC2E5D6A9
:1027A00091E09827F801908385E08093B52024E09C
:1027B00030E0C9012E96CDBFDEBFDF91CF911F91D2
:1027C0000F91FF90EF90DF90CF90BF90AF909F90D0
:1027D0008F907F906F9008952091B6209091B720B0
:1027E000D8018C91863209F4F1C0823509F4EEC02B
:1027F00020E030E0DECF780152E1D52ED701CC9039
:1028000073D68C25F70181937F01DA94B9F760E1E3
:1028100070E0C801E7D3882309F4C1CF8091FC2080
:10282000882309F4E2C1A1D69AE09827D8019C93A5
:10283000BBCF2091B6209091B720D8018C918632E1
:1028400009F4C4C0823509F4C1C0833909F420C237
:102850001092B52020E030E0ACCFC8011CD6D801E2
:102860001496FC9041D68F25F8018483F5803CD6E0
:102870008F25D80115968C9315971696FC9034D613
:102880008F25F8018683F7802FD68F25D8011796DC
:102890008C93179714962C9114979091B920291323
:1028A0001FCF15962C9115979091BA20291318CF08
:1028B00016962C919091BB20291312CF9091BC2099
:1028C00089130ECFF090BD200FD68F25F80180839D
:1028D000F090BD200F2CF294F0240F2CF694F69477
:1028E000F02405D4F801E058FF4F2F2D30E02F5F82
:1028F0003F4F21FB882480F8912C31E083268825E6
:102900008083F090BE20F0D58F25D80111968C934E
:10291000F090BE200F2CF294F0240F2CF694F69435
:10292000F024E5D3F801EF57FF4F2F2D30E02F5F54
:102930003F4F21FBAA24A0F8B12CB1E0AB268A2599
:102940008083F090BF20D0D58F25F8018283F0904E
:10295000BF200F2CF294F0240F2CF694F694F02460
:10296000C6D3F801EE57FF4F2F2D30E02F5F3F4FBA
:1029700021FBCC24C0F8D12C31E0C3268C258083E8
:10298000F090C020B1D58F25D80113968C93F0908C
:10299000C0200F2CF294F0240F2CF694F694F0241F
:1029A000A6D3F801ED57FF4F2F2D30E02F5F3F4F9B
:1029B00021FB662460F8712CB1E06B2686258083AC
:1029C00085E08093B52020E230E1F3CEF80120834A
:1029D000918382E08093B52020E130E0EACE84E06C
:1029E000D8018C9311961C9282E08093B52020E14F
:1029F00030E0DFCEF8018181882309F47CC2F80140
:102A0000108224E030E0D5CE62E070E0C801EAD266
:102A1000882309F4F6C0F80181818C739081903687
:102A200009F485C26AE370E07B01F0E18F9FE00C5E
:102A3000F11C112464E0CE0107960E94DF0444E0FB
:102A400050E060E070E0CE010B960E94FC0546E08D
:102A500050E0B701CE0101960E94FC058F81809362
:102A6000B92088858093BA2089858093BB208A8588
:102A70008093BC2060E470E089EB90E29AD580916D
:102A8000B9208093BD208091BA208093BE20809190
:102A9000BB208093BF208091BC208093C02060E247
:102AA00070E08DEB90E285D5AE01495F5F4FBE01CE
:102AB000655F7F4FCE0101964ED38F81D8018C93F5
:102AC000888511968C931197898512968C9312970D
:102AD0008A8513968C9384E08093B52020E230E0C1
:102AE00068CE62E070E0C8017DD2882309F409C293
:102AF000D80111962C9111972C738C91803609F482
:102B000019C28AE390E07C01B0E12B9FE00CF11C3C
:102B1000112464E0CE0107960E94DF0444E050E0F7
:102B200060E070E0CE010B960E94FC0546E050E0AC
:102B3000B701CE0101960E94FC058F818093B920D8
:102B400088858093BA2089858093BB208A8580936D
:102B5000BC2060E470E089EB90E22BD58091B92035
:102B60008093BD208091BA208093BE208091BB20AD
:102B70008093BF208091BC208093C02060E270E0F1
:102B80008DEB90E216D584E08093B5208F81F8011B
:102B9000808388858183898582838A858383AE014A
:102BA000495F5F4FBE01655F7F4FCE010196D3D273
:102BB00020E230E0FECD6091C120B0E16B9FB0011A
:102BC000112440E150E082EC90E20E94FC0520914B
:102BD000C2208091C6208095281709F4C4C0C5D4AE
:102BE00096E09827D8019C93DFCD6091C120F0E159
:102BF0006F9FB001112440E150E0C8010E9481069E
:102C000012CEB3D491E09827F801908324E030E00D
:102C1000D0CD62E070E0C801E5D1882391F3D801FE
:102C200011966C91B0E16B9FB001112440E150E02E
:102C3000C8010E94FC0560E170E0C801A4D16801F0
:102C4000E0E8CE0ED11CA12CD801BC904DD48B2530
:102C5000F80181938F010B2CB294B0240B2CB69405
:102C6000B694B02444D22B2D30E02F5F3F4F21FB90
:102C7000EE24E0F8F12CF1E0EF268E25D6018D93BD
:102C80006D01A394B2E1AB12DFCF20E930E191CD29
:102C900044E050E060E070E0CE0101960E94FC0547
:102CA0009091B820D80111968C91803209F42FC1EF
:102CB000803709F09DCDD80112962C911297898109
:102CC000281396CD13962C9113978A81281390CDB3
:102CD00014962C9114978B8128138ACD15962C91DC
:102CE00015978C81281384CD9C9361E070E0C80116
:102CF0004AD183E08093B52028E130E05ACD62E0EC
:102D000070E0C8016FD1882381F0D80111968C91B1
:102D10008093C12086E08093B52027D49AE098273D
:102D2000F801908324E030E044CD1FD491E098274F
:102D3000D8019C9324E030E03CCD62E070E0C80113
:102D400051D1882309F45DCFF80181818093C1209E
:102D500088E08093B52009D49AE09827D8019C9305
:102D600024E030E026CD8091CA20281338CFE091AE
:102D7000C3208091C7208095E81331CF8091CB206C
:102D8000E8132DCF8091C4209091C820909589138D
:102D900026CF9091CC20891322CF3091C5209091DD
:102DA000C920909539131BCF9091CD20391317CF9F
:102DB0004091CE209091CF209095491310CF9091C3
:102DC000D02049130CCF9091D1209095491307CF73
:102DD000D8019C911196FC91119712964C911297E3
:102DE00050E060E070E0BA01552744275F2B492B83
:102DF00013969C91792B90E0A0E0B0E0DC0199273C
:102E000088279E2B822BB32B2091B520283009F4E4
:102E10006DC0273021F4840F951FA61FB71F809324
:102E2000C220C92EDA2EEB2EFF24C092C3208D01C2
:102E3000222733270093C4204B2F55276627772757
:102E40004093C520E82FE095E093C620EC2DE09557
:102E5000E093C720E02FE095E093C820E42FE095B1
:102E6000E093C9208093CA20C092CB200093CC204D
:102E70004093CD2085E08093B52020E030E099CCD0
:102E800062E070E0C801AED0882309F44ECFD801CB
:102E900011968C918093C12087E08093B5203DCF1F
:102EA00062E070E0C8019ED0882309F4AACEF80140
:102EB00081818093C12089E04CCF62E070E0C8013D
:102EC00091D0882309F431CF8091FC20811125CF46
:102ED000D80111966C91B0E16B9FB001112440E1D3
:102EE00050E082EC90E20E94810617CF841B950B84
:102EF000A60BB70B94CF62E070E0C80173D08111CC
:102F0000A7CC81E0D8018C9324E030E052CC8981B9
:102F1000F80180833A8131832B8122839C819383C2
:102F2000832782278927848328E230E042CC60E32C
:102F300070E07ACD80E390E0E6CD44E050E060E0E0
:102F400070E00C94FC05CF93DF931F92CDB7DEB7F2
:102F5000FC012181308123273281232733812327DC
:102F6000298344E050E060E070E00E94810641E087
:102F700050E064E070E0CE0101960E9481060F905F
:102F8000DF91CF9108956115710541F1680F791FA7
:102F9000FC0123E633E64191422750E1459FC00101
:102FA0001124A42FA8278A2F90E0582F4427880F98
:102FB000991F880F991F880F991F48275927232F7A
:102FC000332724273527A295AF702A27E617F7075E
:102FD00011F7922F832F908381830895FC0183E65C
:102FE00093E6F9CF61157105B1F1680F791FFC0106
:102FF00023E633E64191422750E1459FC001112469
:10300000A42FA8278A2F90E0582F4427880F991FB4
:10301000880F991F880F991F48275927232F332777
:1030200024273527A295AF702A27E617F70711F74F
:10303000A9015527808190E08417950711F080E061
:103040000895418150E0232F332781E04217530731
:10305000B9F380E0F5CFFC0143E650E023E633E628
:10306000E9CFCF93B091D520C091D6204091D72001
:10307000A091D220F091D320E091D4209C2F907188
:103080002B2F217E9227242F207292272A2F2479FA
:1030900092272F2F237792272E2F2A739227392FAB
:1030A00032953F703927232F269526952327922F77
:1030B000969550E060E070E0BA01552744275C2BFC
:1030C0004B2B769567955795479592279170981356
:1030D0006068A093D520F093D620E093D72040934A
:1030E000D2205093D3206093D420CF910895CF93D2
:1030F000DF93C091D3209091D420A92FAF70B0E07E
:10310000A05EBF4DEC2FEF70F0E0E05EFF4DD0967B
:103110008C912089822BE091D220E295EF70F0E033
:10312000E05EFF4D2081822BC295CF70D0E0C05E63
:10313000DF4D28A1822B92959F70A92FB0E0A05A55
:10314000BF4D9C91892BE82FF0E0E059FF4D808125
:10315000DF91CF910895CF92DF92EF92FF920F937C
:103160001F93CF93DF93FC01DB01EA01918180E0A3
:103170002081822B80FD8DC130E081FD88C120E05F
:103180009695879596958795432F406880FD342FB7
:10319000422F406881FD242F9695879596958795B7
:1031A00036952695432F406880FD342F422F406886
:1031B00081FD242F9695879596958795369526952A
:1031C000432F406880FD342F422F406881FD242F1B
:1031D000969587959695879536952695432F4068C1
:1031E00080FD342F422F406881FD242F96958795CE
:1031F0009695879536952695432F406880FD342F08
:10320000422F406881FD242F969587959695879546
:1032100036952695432F406880FD342F422F406815
:1032200081FD242F969587959695879536952695B9
:10323000532F5068422F406880FD352F3093D520A2
:1032400081FD242F2093D220938180E02281822B44
:1032500080FD1BC130E081FD16C120E09695879569
:1032600096958795432F406880FD342F422F406804
:1032700081FD242F96958795969587953695269569
:10328000432F406880FD342F422F406881FD242F5A
:10329000969587959695879536952695432F406800
:1032A00080FD342F422F406881FD242F969587950D
:1032B0009695879536952695432F406880FD342F47
:1032C000422F406881FD242F969587959695879586
:1032D00036952695432F406880FD342F422F406855
:1032E00081FD242F969587959695879536952695F9
:1032F000432F406880FD342F422F406881FD242FEA
:10330000969587959695879536952695532F50686F
:10331000422F406880FD352F3093D62081FD242F29
:103320002093D320958180E02481822B80FDA9C049
:1033300030E081FDA4C020E096958795969587950D
:10334000432F406880FD342F422F406881FD242F99
:10335000969587959695879536952695432F40683F
:1033600080FD342F422F406881FD242F969587954C
:103370009695879536952695432F406880FD342F86
:10338000422F406881FD242F9695879596958795C5
:1033900036952695432F406880FD342F422F406894
:1033A00081FD242F96958795969587953695269538
:1033B000432F406880FD342F422F406881FD242F29
:1033C000969587959695879536952695432F4068CF
:1033D00080FD342F422F406881FD242F96958795DC
:1033E0009695879536952695532F5068422F4068BD
:1033F00080FD352F3093D72081FD242F2093D420BA
:10340000898111969C9111978927CA8012969C9167
:103410001297C926D12CE12CF12C7601DD24CC2485
:10342000D82A88819C918927C82A8B8113969C91E0
:103430008927F82A10E25BDE082F8C2D817011DEBF
:10344000F694E794D794C794002311F06894F7F8A2
:10345000115089F788818C25888389818D258983FE
:103460008A818E258A838B818F258B83DF91CF91F3
:103470001F910F91FF90EF90DF90CF90089520E47F
:103480005BCF30E456CF20E4E9CE30E4E4CE20E454
:1034900077CE30E472CECF92DF92EF92FF92CF934D
:1034A000FC018181C280D12CE12CF12C7601DD243C
:1034B000CC24D82A8081C82A8381F82AC0E217DE6A
:1034C000B701A60141705527662777278427C9DDF4
:1034D000F694E794D794C794C15089F7CF91FF90A1
:1034E000EF90DF90CF900895CF93DF9300DEC82F49
:1034F00080E0B7DDCC2309F436C0C0E8F8DDD82F72
:1035000080E0AFDDC695D111C068F1DDD82F80E035
:10351000A8DDC695D111C068EADDD82F80E0A1DD15
:10352000C695D111C068E3DDD82F80E09ADDC6953D
:10353000D111C068DCDDD82F80E093DDC695D111B4
:10354000C068D5DDD82F80E08CDDC695D111C0686C
:10355000CEDDD82F80E085DD8C2F8695D111806857
:10356000DF91CF910895C0E0C9CFCF93DF93BFDD46
:10357000C82F80E076DDCC23D1F0C8E0B8DDD82FAD
:1035800080E06FDDC695D111C860B1DDD82F80E035
:1035900068DDC695D111C860AADDD82F80E061DD55
:1035A0008C2F8695D1118860DF91CF910895C0E06E
:1035B000E5CF6F927F928F929F92AF92BF92CF9200
:1035C000DF92EF92FF920F931F93CF93DF933C0113
:1035D000CB010197672BC9F1F301A281C081B181B1
:1035E000D3812A2F2D72322F32953F703227232F0D
:1035F000269526952327322F36954D2F50E060E0F3
:1036000070E0742F6627552744275B2B4C2B6A2BC1
:103610007695679557954795322730FD7068C42F8A
:10362000852E962EA72EBB24B82D6B01EE24FF24E9
:10363000AC2D072F112722273327D02F019788F68B
:10364000F30140838182C2820383DF91CF911F9176
:103650000F91FF90EF90DF90CF90BF90AF909F9031
:103660008F907F906F9008950F931F93CF93DF9368
:10367000CDB7DEB7EC97CDBFDEBF2BD3809315233C
:1036800028D38093162325D38093172322D38093A6
:1036900018231FD3809319231CD380931A2319D383
:1036A00080931B2316D380931C230E94360BB0D328
:1036B000882389F09091152380911623853009F491
:1036C00052C0B0F0883009F4B3C0893009F498C012
:1036D000863009F45AC09CD3882311F06DD350D39F
:1036E000EC96CDBFDEBFDF91CF911F910F91089572
:1036F000813021F008F468C0833069F7992309F418
:10370000A1C0923041F780911723811127C0009109
:10371000192310911A230F70112701151105D9F2E1
:10372000802FF5D280911623833009F4E6C0E09112
:103730001F23F091202381818B7F818384E8809FE8
:10374000F001819FF00D1124ED59FC4D1082E091A4
:103750001F23F091202380818E7F808380E0D7D249
:103760002BD38FD4B8CF9111B6CF109117231F77D9
:1037700023D387D47FD38823E9F31093C304111193
:1037800076C082E080931423A6CF9058923008F040
:10379000A2CF80911723909118238C3D23E09207AC
:1037A00009F467C0AE01455C5F4F609119230E9428
:1037B00088038C01009709F48ECFFED2B8018BAD3F
:1037C0009CADC0D177D287CF903809F447C09238EA
:1037D00009F081CF809119238F7099D2E0911F2336
:1037E000F0912023118112FB112710F980E08FD274
:1037F000E3D2812F7DD280E07BD243D242D46BCF03
:10380000911169CF80911723823008F064CFD4D210
:10381000809117238093102334D480911023882320
:1038200009F461C084E0809314230E94320B53CFCB
:10383000903809F050CFC0D28091102359D221D2B4
:1038400020D449CF90911723913009F044CF91E0D3
:10385000833009F090E09093122380CF10911123D0
:1038600080911223882309F4C3CF1260C1CF83E073
:1038700089CF83E08A838AE389835FB7F89482E003
:103880008093CA01E8E0F0E0E4911092CA01DE0101
:10389000139620E038E042E0EF708E2F90E0EA309F
:1038A000B8F0C7968D939D932F5F2C3199F040937C
:1038B000CA01E32FF0E0E4911092CA0120FFECCF9F
:1038C000E295EF703F5FEF708E2F90E0EA3048F79F
:1038D000C096E8CF5FBF70D26AE370E0CE01019678
:1038E00090D0E8D1F8CE8091C304882321F084E001
:1038F000809314239ACF81E0FBCF42D22FCF08953B
:10390000CF9380911423811102C0CF910895C0916B
:10391000212380E0FCD17CD2811103C08C2FCF9178
:10392000F6C1A2DE8C2FCF91F2C1AF92BF92DF928F
:10393000EF92FF920F931F93CF93DF938C01EB01D4
:103940007A01B5D3D82E811127C0E114F104A1F179
:10395000F70120813181C21BD30B020F131F209767
:10396000D9F0A12CB12C80911D2390911E23FC0134
:10397000EF5BFF4F2081FC01E05CFF4F8081281747
:1039800090F17FD1BDDFF701808191818A0D9B1D70
:103990008083918325E0D22E8D2DDF91CF911F91D1
:1039A0000F91FF90EF90DF90BF90AF90089569D195
:1039B000A7DF7DD3811123C0209771F320911D23B0
:1039C00030911E23F901EF5BFF4F9081F901E05C1C
:1039D000FF4F8081981758F7F80181918F0188D1A6
:1039E000219761F7D9CFF80181918F0181D1FFEF44
:1039F000AF1ABF0ACA15DB0509F0B5CFCDCFD82E57
:103A0000CBCFCF92DF92EF92FF920F931F93CF9382
:103A1000DF936C01EB0180912123806878D10091C4
:103A20001B2310911C230C171D0720F0209709F46D
:103A300083C08E01C0E00115110509F04AC0CC23F6
:103A400009F45CC080911423882309F455C08530A3
:103A500009F45DC0DDD181116DC0F3D181114EC07B
:103A600009D2882379F38091212387FD5AC02091C0
:103A70001D2330911E23F901E05CFF4FE080F90126
:103A8000EF5BFF4F8081F12CE81AF1080115110559
:103A9000A9F088E0E816F10488F4E60104C088E0A3
:103AA000E816F10459F0899123D16E0101501109F2
:103AB0008FEFE81AF80A0115110589F7C1E088E0CF
:103AC000E816F10409F0C0E0DCD00115110509F495
:103AD000B6CF80911423882379F08530C1F098D136
:103AE000811128C0AED1811109C0C4D18111BBCFD1
:103AF000809114238111F1CF82E00AC0A2D18111FB
:103B00001FC0809114238823B9F38530B9F783E06F
:103B1000DF91CF911F910F91FF90EF90DF90CF90A9
:103B20000895E0911D23F0911E23EF5BFF4FE0808D
:103B3000F12CACCF81E0ECCFA4D000E010E07ACF44
:103B400080E0E6CFCF92DF92EF92FF920F931F9328
:103B5000CF93DF93D82EC92E8B01809121238068CB
:103B6000D6D0C0911B23D0911C23C017D10728F0B9
:103B70000115110509F47FC0E801ED2CFC2CD12CB6
:103B8000209709F045C0DD2009F457C08091142327
:103B9000882309F450C0853009F458C039D1811107
:103BA00068C04FD1811149C065D1882379F38091D4
:103BB000212387FD55C080911D2390911E23FC0178
:103BC000E05CFF4F0081FC01EF5BFF4F808110E064
:103BD000081B1109209791F00830110520F00EC044
:103BE0000830110559F0F701849182D0FFEFEF1AE8
:103BF000FF0A21970F5F1F4F209791F7DD24D39481
:103C00000830110509F0D12C3CD0209709F4BBCF26
:103C100080911423882379F08530C1F0F9D0811187
:103C200028C00FD1811109C025D18111C0CF809149
:103C300014238111F1CF82E00AC003D181111FC08A
:103C4000809114238823B9F38530B9F783E0DF919D
:103C5000CF911F910F91FF90EF90DF90CF9008953B
:103C6000E0911D23F0911E23EF5BFF4F008110E0D8
:103C7000B1CF81E0ECCF05D0C0E0D0E07ECF80E0D6
:103C8000E6CFE0911F23F0912023A0911D23B09156
:103C90001E23AF5BBF4F8C9190E082839383808122
:103CA0008D798083E0911D23F0911E23EF5BFF4F00
:103CB00010820895E0911F23F091202380818D7957
:103CC0008083E0911D23F0911E23EF5BFF4F108254
:103CD000089580911D2390911E23FC01EF5BFF4FFF
:103CE0002081DC01A20FB11D8C912F5F20830895EC
:103CF00020911D2330911E23F901EF5BFF4F90812E
:103D0000D901A90FB11D8C939F5F90830895809373
:103D10002123282F2F70622F70E094E8299F9001B3
:103D200011242E5D3C4D4091C6045091C70487FD7F
:103D300012C020931D2330931E23CB0182959295B0
:103D4000907F9827807F9827840F951F80931F234B
:103D50009093202308952E5B3F4F20931D23309393
:103D60001E2362957295707F7627607F7627685F45
:103D70007F4F640F751F60931F2370932023089556
:103D8000E0911F23F0912023818184608183E09161
:103D90001F23F09120238181807C803409F00895D5
:103DA000809121238058B3DFE0911F23F0912023DD
:103DB0008181846081830895809121238F77A7DF9B
:103DC000E0911F23F091202380818D788083E09102
:103DD0001F23F0912023808181608083E0911D2347
:103DE000F0911E23EF5BFF4F1082809121238068AA
:103DF0008EDFE0911F23F0912023808181608083FA
:103E0000E0911D23F0911E23EF5BFF4F1082089578
:103E1000809121238F777BDFE0911F23F091202376
:103E2000808184FF0CC020911D2330911E2382814C
:103E30009381F901E05CFF4F808381E0089580E089
:103E40000895809121238F7762DFE0911F23F09105
:103E50002023808185FF0CC020911D2330911E23DB
:103E600082819381F901E05CFF4F808381E00895B6
:103E700080E0089580912123806849DFE0911F232D
:103E8000F091202380818695817008951F93CF93B0
:103E9000DF9300D0CDB7DEB7182F4A83698337DFB1
:103EA000E0911F23F09120231182E0911F23F091D4
:103EB00020234A81698117FD22C01082E0911F23CF
:103EC000F09120236183E0911F23F091202312823F
:103ED000138280911D2390911E238483958340E05B
:103EE000FC01E05CFF4F4083FC01EF5BFF4F108261
:103EF00081E00F900F90DF91CF911F91089582E0A4
:103F00008083E0911F23F09120236183E0911F23A0
:103F1000F09120231282138280911D2390911E2301
:103F200084839583DDCFAF92BF92DF92EF92FF92B1
:103F30000F931F93CF93DF9300D0CDB7DEB7E62E5C
:103F4000662309F44AC05C018C010C5F1F4FF12C01
:103F5000D5015C915523C9F1D5011196ED91FC91E4
:103F60001297D80111974C91D8018C91823008F4A6
:103F700043C098E188E1E930F10550F028E030E0F5
:103F800090E09F5F220F331F2E173F07D0F3982B2F
:103F9000252F2F7030E02630310564F5E134F1052E
:103FA00048F59F7E41112BC09064DE2E4E2F692F65
:103FB000852F805859839A8369DF9A8159814D2DC5
:103FC000692F852F63DF8823A9F0F394B5E0AB0E4A
:103FD000B11C0B5F1F4FFE10BBCF81E00F900F9005
:103FE000DF91CF911F910F91FF90EF90DF90BF90E5
:103FF000AF90089580E0F2CF98E088E0BCCF4130E8
:1040000029F09068442389F2DE2ED9CF906CDE2E01
:10401000D6CFE0ECF4E0A681B78119961C92A68178
:10402000B78111961C92A681B78159961C92A681E0
:10403000B78151961C92A681B78199961C92A68150
:10404000B78191961C92A681B781D9961C92A681C0
:10405000B781D1961C92A681B781A75BBF4F1C92F6
:10406000A681B781AF5BBF4F1C92A681B781A75ACB
:10407000BF4F1C920680F781E02DEF5AFF4F108250
:1040800008958091152387FD08C0F4DE81110DC0CD
:10409000809114238111F9CF0895D3DE811106C0D8
:1040A000809114238111F9CF0895EBCD03CE1F9396
:1040B000CF93DF93E091C604F091C704E05AFF4F1D
:1040C000C081D18114E6809121238078803831F13C
:1040D000B8DE811126C080911423882339F1853000
:1040E00051F1E0911F23F0912023818182FD28C0AE
:1040F000E091C604F091C704E05AFF4F808191819E
:10410000C817D90701F3212F21501123F1F0EC0139
:10411000122F8091212380788038D1F6ABDE88235E
:10412000D1F280E0DF91CF911F91089582E0DF917D
:10413000CF911F91089583E0DF91CF911F91089552
:1041400081E0DF91CF911F91089584E0DF91CF91BD
:104150001F91089563D069D0E0ECF4E081818E7FF7
:10416000818380818F778083109213230895CF936A
:10417000DF93E0E4F0E014828481816084834ED098
:1041800054D0C0ECD4E088818F77888388818068A0
:1041900088831092142310921023109212231092ED
:1041A000112388818064888348E068E480E86EDEBB
:1041B00048E068E480E06ADE8885806488878981D9
:1041C00081608983DF91CF910895CF93DF933FB7CB
:1041D000F894C0ECD1E022E02A87EAE1F0E0E49133
:1041E000A0ECB4E0DA96EC93DA97EBE1F0E0E4913E
:1041F000DB96EC93DB971A868BE396E28E7F16961E
:104200008D939C93179785E18C9318962C933FBFC1
:1042100081E080931323DF91CF91A9CFE0ECF4E00C
:1042200080858370808711860895E0ECF4E08FEF3D
:104230008287848708951F920F920FB60F921124E0
:104240002F933F934F935F936F937F938F939F939E
:10425000AF93BF93EF93FF938091CA0487FD4DC046
:104260008091CA0486FD41C08091CA0485FF0CC0BC
:1042700080E28093CA0480911023882371F184E046
:10428000809314230E94280B8091CA0484FF14C0D9
:1042900080E18093CA0482E080931423109210235B
:1042A0001092C304B6DE48E068E480E8EFDD48E041
:1042B00068E480E0EBDD23DBFF91EF91BF91AF91EC
:1042C0009F918F917F916F915F914F913F912F912E
:1042D0000F900FBE0F901F9018958091C30481110D
:1042E00015C081E080931423CDCF80E48093CA046D
:1042F000109214230E942D0BB7CF8091C80487FF22
:10430000AFCF80E88093CA04FADAAACF83E0EACF7D
:10431000CF93DF93EC014096FC018BE0DF011D920F
:104320008A95E9F782E08C83898783E08E8761E054
:10433000CE010196F8DD811104C080E0DF91CF91BC
:10434000089561E0CE010696EEDD8823B1F361E0C9
:10435000CE010B96DF91CF91E6CDCF93DF93D62F91
:10436000C72F20911423243021F082E0DF91CF91D8
:104370000895FC014489558966897789452B462B28
:10438000472B99F38181C3DCAD2FBC2FFD01019038
:104390000020E9F7BF01615071096A1B7B0B40E007
:1043A00050E08D2F9C2FDF91CF91BFCAEF92FF92EB
:1043B0000F931F93CF93DF93EB017A012091142386
:1043C000243041F082E0DF91CF911F910F91FF9057
:1043D000EF900895FC010489158926893789012BFE
:1043E000022B032B79F3818192DC40E050E0B7018E
:1043F000CE01DF91CF911F910F91FF90EF9095CA61
:104400000F931F93CF93DF931F92CDB7DEB7209109
:104410001423243039F082E00F90DF91CF911F9167
:104420000F910895FC010489158926893789012B8C
:10443000022B032B81F38181698369DC20911D2389
:1044400030911E23F901EF5BFF4F9081F901E05C91
:10445000FF4F80816981981730F0698312DC27DE75
:1044600069818111D9CF862F43DC80E0D5CF0F93AE
:104470001F93CF93DF931F92CDB7DEB72091142304
:10448000243039F082E00F90DF91CF911F910F918E
:104490000895FC014489558966897789452B462B07
:1044A000472B81F3818133DC8091212320911D23CF
:1044B00030911E23F90187FD1DC0E05CFF4F808114
:1044C000F901EF5BFF4F408190E0841B9109892B3C
:1044D00011F480E0D8CF0081F901E05CFF4F10813A
:1044E000D0DB0117B0F3E3DD8111CDCF8983C9DBC8
:1044F0008981C9CFEF5BFF4F808190E0E8CFCF93F8
:10450000DF93EC0180911423843019F0DF91CF9177
:1045100008954C895D896E897F89452B462B472BF1
:10452000A9F38981F4DBA6DC882381F3CE01DF9136
:10453000CF919DCFCF93DF93209114232430C1F5E9
:10454000FC014489558966897789452B462B472B81
:1045500079F18681DCDB75DC882351F180912123A0
:1045600087FD3DC080911D2390911E23FC01E05CDE
:10457000FF4F2081FC01EF5BFF4F408130E0241BA7
:104580003109232BD9F4CFEFDFEF2091212327FD31
:1045900023C0DC01A05CBF4F8C91208190E0821B86
:1045A0009109892B39F486DBCE01DF91CF910895F3
:1045B000CFEFDFEFCE01DF91CF9108958ADBC82FD7
:1045C000D0E080911D2390911E23FC01EF5BFF4FF3
:1045D0002091212327FFDDCF808190E0E2CF8091E1
:1045E0001D2390911E23FC01EF5BFF4F208130E0E3
:1045F000C8CF0895FF920F931F93CF93DF93EC01E1
:1046000007DC882349F0888190E0209119233091BC
:104610001A232817390731F0DF91CF911F910F919D
:10462000FF90089580911623813209F44BC008F061
:1046300033C0803289F780911523813269F7BCDB62
:1046400004C080911423882339F3FBDB8823C9F34A
:1046500040DB082F3EDB182F3CDBF82E3ADB4F2DDA
:1046600050E060E070E0BA0155274427782B402BDA
:10467000512B4C8B5D8B6E8B7F8B2BDB888F29DBDB
:10468000898F27DB8A8F16DBFCDCCE01DF91CF918F
:104690001F910F91FF90ADCF823209F434C0833265
:1046A00009F0BACF80911523813209F0B5CF84DBB0
:1046B000E8DC60911723CE01DF91CF911F910F911C
:1046C000FF9097CF80911523813A09F0A5CF74DB35
:1046D000D1DB8823E9F38C89FD880E891F8908DBEB
:1046E0008F2D06DB802F04DB812F02DB888D00DB22
:1046F000898DFEDA8A8DFCDAC4DADF91CF911F91C1
:104700000F91FF90BECC80911523813209F084CFA8
:1047100053DBB7DC8091172390911823888B998BFA
:10472000CE01DF91CF911F910F91FF9062CFB7FF24
:1047300004C003D0821B930B089509D0A59F900D50
:10474000B49F900DA49F800D911D11240895A29FE8
:10475000B001B39FC001A39F01D0B29F700D811D16
:104760001124911D08958F929F92AF92BF92CF9284
:10477000DF92EF92FF92CF93DF93EC016881798112
:104780008A819B81611571058105910521F464E29F
:1047900079ED8BE597E02DE133EF41E050E038D340
:1047A00049015A019B01AC01A7EAB1E4C6DF6B01E4
:1047B0007C01ACEEB4EFA5019401BBDFC60ED71EA1
:1047C000E81EF91EF7FE06C081E0C81AD108E1080C
:1047D00080E8F80AC882D982EA82FB82E894D7F896
:1047E000EE24FF24C601DF91CF91FF90EF90DF9080
:1047F000CF90BF90AF909F908F900895B4CF8CE1F1
:1048000090E2B1CFA0E0B0E080931C2090931D20F7
:10481000A0931E20B0931F200895FB01DC0102C06D
:1048200005900D9241505040D8F70895FB01DC01EE
:104830008D91059080190110D9F3990B0895FB0112
:10484000DC014150504048F005900D920020C9F71E
:1048500001C01D9241505040E0F70895FB01DC017A
:1048600002C001900D9241505040D8F70895AEE03B
:10487000B0E0ECE3F4E2F5C20D891E898F89988DD2
:104880002EE02C8309831A8397FF02C080E090E812
:1048900001978D839E83CE014B96AC01698D7A8DF5
:1048A000CE01019611D04D815E8157FD0AC02F8146
:1048B0003885421753070CF49A01F801E20FF31FF1
:1048C00010822E96E4E0E6C2ACE0B0E0E9E6F4E265
:1048D000BAC27C016B018A01FC01168217828381B6
:1048E00081FFB9C188248394912C8C0E9D1EF70101
:1048F0009381F60193FD859193FF81916F01882348
:1049000009F4A5C1853239F493FD859193FF819116
:104910006F01853221F4B70190E0F0D1E8CF512C3E
:10492000312C20E02032A8F48B3261F028F4803260
:1049300051F0833271F40BC08D3239F0803349F479
:10494000216028C02260246025C0286023C0206127
:1049500021C027FD27C0382F30533A3078F426FF86
:1049600006C0FAE05F9E300D1124532E13C08AE07A
:10497000389E300D1124332E20620CC08E3221F46B
:1049800026FD65C1206406C08C3611F4206802C083
:10499000883641F4F60193FD859193FF81916F0173
:1049A0008111C0CF982F9554933018F090529330C6
:1049B00028F40C5F1F4FFFE3F9830DC0833631F0FD
:1049C000833771F0833509F05AC022C0F801808125
:1049D00089830E5F1F4F44244394512C540114C00B
:1049E0003801F2E06F0E711CF801A080B18026FF43
:1049F00003C0652D70E002C06FEF7FEFC5012C870B
:104A000072D12C0183012C856FE7262E222217C03C
:104A10003801F2E06F0E711CF801A080B18026FF12
:104A200003C0652D70E002C06FEF7FEFC5012C87DA
:104A30004FD12C012C8550E8252E222A830123FCFE
:104A40001AC005C0B70180E290E058D13A94832D96
:104A500090E048165906B0F30EC0F50127FC859189
:104A600027FE81915F01B70190E048D131103A945F
:104A7000F1E04F1A51084114510479F7E5C084362A
:104A800011F0893639F5F80127FF07C0608171817F
:104A9000828193810C5F1F4F08C0608171818827DC
:104AA00077FD8095982F0E5F1F4F4FE6B42EB222F0
:104AB00097FF09C090958095709561957F4F8F4FB6
:104AC0009F4FF0E8BF2A2AE030E0A40143D1A82E8E
:104AD000A81842C0853731F43FEEB32EB2222AE047
:104AE00030E024C099EFB92EB2228F36B9F020F40D
:104AF000883509F0ACC00DC0803721F0883709F047
:104B0000A6C002C020E1B22AB4FE0BC084E0B82ADD
:104B100008C024FF09C0E6E0BE2A06C028E030E055
:104B200005C020E130E002C020E132E0F801B7FE2C
:104B300007C060817181828193810C5F1F4F06C025
:104B40006081718180E090E00E5F1F4FA40102D16F
:104B5000A82EA818FFE7BF22B6FE0BC02B2D2E7F74
:104B6000A51450F4B4FE0AC0B2FC08C02B2D2E7E52
:104B700005C07A2C2B2D03C07A2C01C0752C24FF84
:104B80000DC0FE01EA0DF11D8081803311F4297EF4
:104B900009C022FF06C07394739404C0822F8678E4
:104BA00009F0739423FD13C020FF0EC05A2C731418
:104BB00058F4530C5718732C07C0B70180E290E0EB
:104BC0002C879CD073942C857314B8F304C0731491
:104BD00010F4371801C0312C24FF11C0B70180E355
:104BE00090E02C878BD02C8522FF1CC021FF03C0B6
:104BF00088E590E002C088E790E0B7010CC0822F02
:104C0000867881F021FD02C080E201C08BE227FDA1
:104C10008DE2B70190E072D005C0B70180E390E06B
:104C20006DD05A94A514C8F3AA94F401EA0DF11DAD
:104C3000B701808190E062D0A110F6CF05C0B70126
:104C400080E290E05BD03A943110F9CF50CEF7017A
:104C50002681378102C02FEF3FEFC9012C96E2E198
:104C60000BC1E0ECF1E0A785A7FDFDCFA485A8600E
:104C7000A4876050704FF2CDDC01CB0102C02D91B2
:104C800005D041505040D8F70895262FE0ECF1E0D0
:104C9000378537FDFDCF3485377F3487378531FF42
:104CA00009C036E3328738ED34BF31E033873785CA
:104CB00037FDFDCF33E332878083918312822483D3
:104CC00025E3228728ED31E024BF3387019608953C
:104CD000FC010590615070400110D8F780959095C7
:104CE0008E0F9F1F0895FC016150704001900110CC
:104CF000D8F7809590958E0F9F1F08950F931F935F
:104D0000CF93DF938C01EB018B8181FD03C00FEF0B
:104D10001FEF1AC082FF0DC02E813F818C819D81C3
:104D20002817390764F4E881F9810193E883F9834E
:104D300006C0E885F985802F0995892B41F78E817A
:104D40009F8101968E839F83C801DF91CF911F9130
:104D50000F910895FA01AA27283051F1203181F1ED
:104D6000E8946F936E7F6E5F7F4F8F4F9F4FAF4F73
:104D7000B1E03ED0B4E03CD0670F781F891F9A1F86
:104D8000A11D680F791F8A1F911DA11D6A0F711D3A
:104D9000811D911DA11D20D009F468943F912AE046
:104DA000269F11243019305D3193DEF6CF0108952E
:104DB000462F4770405D4193B3E00FD0C9F7F6CF5F
:104DC000462F4F70405D4A3318F0495D31FD405227
:104DD000419302D0A9F7EACFB4E0A69597958795BD
:104DE00077956795BA95C9F700976105710508959C
:104DF0009B01AC010A2E0694579547953795279548
:104E0000BA95C9F7620F731F841F951FA01D0895DF
:104E1000052E97FB16F4009406D057FD0CD044D015
:104E200007FC09D07EF490958095709561957F4F31
:104E30008F4F9F4F089550954095309521953F4F46
:104E40004F4F5F4F08952F923F924F925F926F9214
:104E50007F928F929F92AF92BF92CF92DF92EF920A
:104E6000FF920F931F93CF93DF93CDB7DEB7CA1B8B
:104E7000DB0BCDBFDEBF09942A88398848885F8460
:104E80006E847D848C849B84AA84B984C884DF80EA
:104E9000EE80FD800C811B81AA81B981CE0FD11DCE
:104EA000CDBFDEBFED010895A1E21A2EAA1BBB1BE8
:104EB000FD010DC0AA1FBB1FEE1FFF1FA217B307E6
:104EC000E407F50720F0A21BB30BE40BF50B661FFC
:104ED000771F881F991F1A9469F7609570958095C0
:104EE00090959B01AC01BD01CF010895F894FFCFCF
:104EF000008310000001041000000182080000017E
:104F0000000000000000000000000014010000008C
:104F10000001010100000001000001000101000189
:104F20000000000202000002000202020200000271
:104F30000000000404000004000404040400000451
:104F40000008080800000008000008000808000821
:104F500000000010100000100010101010000010D1
:104F6000000100010000000000000001000101013B
:104F70000101010001000100000001010001010127
:024F800000002F
:00000001FF
